:04000000B601062916
:1000080008009818181218162C08A0002D08A1002E
:10001800A201A3010F28102864008C1A2C28FF3095
:10002800A207031CA307031CA007031CA107031CAA
:100038000129220F0E28230F0F28FA30A2000030C2
:10004800A300102898181812181664008C1E292866
:100058001A080314012964000C1E2F2899000314A0
:100068000129B616B61EB612B6193E28B61577205F
:10007800031865280830A3008B20A20DA30B402885
:10008800B61E702095209120B61A65206A20220895
:1000980003100129B616B61EB61236195828FE39AD
:1000A800B700361503100129361A6028A60036163F
:1000B80077200318652826087E2003186528B61EB1
:1000C80001297020952036113612B6113A0884009D
:1000D80038088417800476283A088400380980058F
:1000E8008417800508006A20952070209120370821
:1000F800B6190138A2000830A300A20D03186A201F
:10010800031C702095209120A30B81286A2095203C
:100118003A08840038080005FF3E3B088400390986
:1001280073283B08840039086D28A40029080314A3
:1001380003190129FC20031C0800A00025188317B7
:1001480024088400200880008313A40AA9039A289D
:10015800A301A200FF30A207031CA307031C012967
:100168000330A100E630BA20AE28A101FC3EA00071
:10017800A109031CC528FF300000A0070318C028E8
:10018800A0076400A10FBF2808000310A00DA10D4F
:10019800FF3E0318C92820080129A2000130D628EB
:1001A800A2000530A80023082102031DDD2822082B
:1001B8002002043003180130031902302805031DFA
:1001C800FF3001291030A800A101A001A70CA60C3E
:1001D800031CF4282208A00723080318230FA107EB
:1001E800A10CA00CA50CA40CA80BEA282408012932
:1001F800840031088A0030088200831303138312B5
:100208006400080083160F3099002030980083128C
:1002180090309800831607309F00D701D8018312C9
:100228008712831687128801071087100711871213
:100238008901831287128316871283120710831687
:1002480007100A3083128A01AC200714831607109E
:1002580083120130A3002C308A01AD2053308A016B
:100268002F2074308A012F2061308A012F207230AC
:100278008A012F2074308A012F2069308A012F20AB
:100288006E308A012F2067308A012F202E308A0194
:100298002F202E308A012F208A110A12742B09115F
:1002A800831609114208831288008A110A126229EA
:1002B800091583160911440883128800071183164B
:1002C80007118312000000000000000007158316C4
:1002D8000711831209118316091183120800831666
:1002E8004630C40083128A015C218316C20183123E
:1002F8008A01532183161030C20083128A015321C8
:1003080083164C30C40083128A015C218316423064
:10031800C40083128A015C218316C2010130C60021
:10032800831264008130831646028A110A128312EE
:100338000318BB2983160130C900831264002130D9
:10034800831649028A110A1283120318B4298A01F2
:1003580053218316C90A8A110A128312031DA2297E
:100368008316C60A8A110A128312031D9529831659
:100378004630C40083128A015C218316C2018312AD
:100388008A01532183161030C20083128A01532137
:1003980083164C30C40083128A015C21080083163E
:1003A8004630C40083128A015C218316C20183127D
:1003B8008A01532183161030C20083128A01532107
:1003C80083164C30C40083128A015C21080083160E
:1003D8004630C40083128A015C218316C20183124D
:1003E8008A0153218316C20183128A01532183167D
:1003F8004C30C40083128A015C2183164230C40049
:1004080083128A015C2183160130C60083126400BE
:100418001130831646028A110A1283120318352AEC
:1004280083160130C9008312640021308316490203
:100438008A110A12831203182E2A83162030C2004A
:1004480083128A0153218316C90A8A110A12831258
:10045800031D182A8316C60A8A110A128312031D5D
:100468000B2A83164630C40083128A015C21831646
:10047800C20183128A0153218316C2014C30C40081
:1004880083128A015C21080083164030C40083125D
:100498008A015C218316C601831264000830831622
:1004A80046028A110A1283120318822A8316460802
:1004B800073C8A110A128312031C792A8A110A122C
:1004C8006B228316C20083128A110A12792A02301B
:1004D8008A0083164608831282073034873407342B
:1004E8001F3452347F34203400348A015321831658
:1004F800C60A8A110A128312031D512A8316443030
:10050800C40083128A015C218316C6018312640029
:100518000630831646028A110A1283120318BA2A71
:1005280083164608053C8A110A128312031CB12A55
:100538008A110A12A5228316C20083128A110A128E
:10054800B12A02308A0083164608831282070034D3
:1005580000347F34003410347F348A0153218316E9
:10056800C60A8A110A128312031D8B2A83165A306F
:10057800C40083128A015C218316C20183128A0196
:10058800532183165B30C40083128A015C218316D1
:100598000130C20083128A01532183165830C400E7
:1005A80083128A015C2183161630C20083128A01E5
:1005B80053218A0173218A01EB2183164630C40036
:1005C80083128A015C218316C20183128A01532196
:1005D8008316C20183128A01532183164C30C4004A
:1005E80083128A015C2183164230C20083128A0179
:1005F80053218316C20183128A01532183165D3069
:10060800C40083128A015C2183160430C20083125D
:100618008A01532183168630C20083128A0153212E
:1006280083165930C40083128A015C218316143062
:10063800C20083128A01532183164C30C4008312EE
:100648008A015C210800831646083C3E84000008A5
:100658008312B200FF30A200A20A22080F3C8A11BE
:100668000A12031C5A2B8A110A12462332028A11D3
:100678000A12031D302B22088316CE0083128A111A
:100688000A125A2B03308A00220882073034313488
:100698003234333434343534363437343834393406
:1006A80041344234433444344534463408008316D4
:1006B8004630C40083128A015C2183162A08C200CE
:1006C80083128A01532183162B08C20083128A01E0
:1006D800532183164508C40083128A015C2108004F
:1006E8008A0148228316A530AA00AB014C30C50008
:1006F80083128A015B2383164230C40083128A0165
:100708005C218316C60183126400163083164602E4
:100718008A110A1283120318C72B83164608153C40
:100728008A110A128312031CBE2B8A110A12A223F1
:100738008316C20083128A110A12BE2B03308A0064
:1007480083164608831282075034493443342034D0
:1007580043346F346E34743472346F346C346C34A4
:1007680065346434203453344534443431343334B8
:10077800333430348A0153218316C60A8A110A1287
:100788008312031D882B8316C630AA00AB014C3098
:10079800C50083128A015B2383164230C40083128A
:1007A8008A015C218316C601831264001330831604
:1007B80046028A110A12831203181D2C8316460852
:1007C800123C8A110A128312031C142C8A110A1271
:1007D800F3238316C20083128A110A12142C0430E0
:0A07E8008A00831646088312002CD5
:100800008207323435343634783431343234383443
:10081000203447347234613470346834693463345A
:1008200020344C34433444348A0153218316C60A9D
:100830008A110A128312031DD92B8316E330AA00F2
:10084000AB014C30C50083128A015B238316423012
:10085000C40083128A015C218316C60183126400DE
:100860001B30831646028A110A1283120318732C56
:10087000831646081A3C8A110A128312031C6A2C3A
:100880008A110A1249248316C20083128A110A129D
:100890006A2C04308A008316460883128207553476
:1008A000733469346E3467342034503469346334BB
:1008B00042346134733469346334503472346F3485
:1008C00020345634653472342E34203432342E348D
:1008D000343432348A0153218316C60A8A110A122B
:1008E0008312031D2F2C83160530AA000130AB00A4
:1008F0004C30C50083128A015B2383164230C4004A
:1009000083128A015C218316C601831264001530AC
:10091000831646028A110A1283120318C42C831606
:100920004608143C8A110A128312031CBB2C8A113C
:100930000A12A0248316C20083128A110A12BB2C49
:1009400004308A00831646088312820752346134C9
:100950006E346A34693474342034443469346F3406
:100960006C3420342D34203443344F344D345034DF
:100970005334793473348A0153218316C60A8A1199
:100980000A128312031D862C83162430AA0001301C
:10099000AB004C30C50083128A015B2383164230C2
:1009A000C40083128A015C218316C601831264008D
:1009B0001730831646028A110A1283120318212D5A
:1009C00083164608163C8A110A128312031C182D3E
:1009D0008A110A12F1248316C20083128A110A12A4
:0E09E000182D05308A00831646088312002D5C
:100A0000820768347434743470343A342F342F3499
:100A10007734773477342E3463346F346D347034F4
:100A200073347934733431342E3463346F346D3429
:100A30008A0153218316C60A8A110A128312031DE2
:100A4000D72C83168230AA000130AB004C30C50091
:100A500083128A015B2383164230C40083128A0109
:100A60005C218316C601831264001B308316460284
:100A70008A110A1283120318782D831646081A3C2D
:100A80008A110A128312031C6F2D8A110A124E2535
:100A90008316C20083128A110A126F2D05308A0054
:100AA0008316460883128207553473346534203424
:100AB0007734693474346834203447344C344334E4
:100AC0004434203454344F344F344C345334203471
:100AD000563465347234203431342E3434348A013F
:100AE00053218316C60A8A110A128312031D342D5C
:100AF0008316AA011030AB004F30C50083128A0163
:100B00005B2383164230C40083128A015C21831662
:100B10008030C200C6018312640080308316460212
:100B20008A110A12831203189E2D8A0153218316FB
:100B3000C60A8A110A128312031D8C2D83161F30D8
:100B4000AA001030AB004F30C50083128A015B232E
:100B500083164230C40083128A015C21831601305F
:100B6000C200C601831264008030831646028A11D7
:100B70000A1283120318C52D8A0153218316C60A4F
:100B80008A110A128312031DB32D8316AA01103095
:100B9000AB004C30C50083128A015B2383164230C0
:100BA000C40083128A015C218316FF30C200C60193
:100BB000831264002030831646028A110A128312BF
:100BC0000318EB2D8A0153218316C60A8A110A12D3
:100BD0008312031DD92D8316E030AA001F30AB000D
:100BE0004C30C50083128A015B2383164230C40057
:100BF00083128A015C218316FF30C200C601831272
:100C000064002030831646028A110A1283120318E8
:100C1000122E8A0153218316C60A8A110A128312E0
:100C2000031D002E8316C901C601CA012030C10070
:100C3000AA01AB01B401B501B601B7017830C70014
:100C4000C801573083128A012F2061308A012F207A
:100C500069308A012F2074308A012F2069308A017F
:100C60002F206E308A012F2067308A012F202E30EE
:100C70008A012F202E308A012F200A308A012F204E
:100C80000D308A012F2011308A012F2011308A0166
:100C90002F2011308A012F208A012620403C8A1102
:100CA0000A12031D4C2E0B30A9002630B000B101F2
:100CB000A501A0308A01992013308A012F2013301A
:100CC0008A012F2013308A012F2013308A012F2010
:100CD0008A01EB218316C601831264000B30831650
:100CE00046028A110A1283120318B52E831646088B
:100CF000A03E840000088312B200FF30A200A20AC6
:100D000022080F3C8A110A12031CA92E8A110A120A
:100D1000952632028A110A12031D7F2E220883169D
:100D2000CE0083128A110A12A92E06308A002208E8
:100D30008207303431343234333434343534363459
:100D4000373438343934413442344334443445340C
:100D5000463483164608A03E84004E088000C60A2A
:100D60008A110A128312031D6D2E83162008C900F2
:100D700021088312A000A10104308A01CC20B20016
:100D80002108B30083162208831232048316C1009F
:100D900023088312A000A10104308A01CC20B200F4
:100DA0002108B30083162408831232048316AB0093
:100DB00025088312A000A10104308A01CC20B200D2
:100DC0002108B30083162608831232048316AA0072
:100DD00027088312A000A10104308A01CC20B200B0
:100DE0002108B30083162808831232048316D0002A
:100DF00029088312A000A10104308A01CC20B2008E
:100E00002108B30083162A08831232048316CF0008
:100E10002B08D1002A08D2002A088312FE0083166C
:100E20002B088312FF00831650088312FD008316DF
:100E30004F088312FC00640083164908003C8A15A1
:100E40000A12831203196629640083164908013CBB
:100E50008A150A128312031964296400831649084B
:100E6000023C8A150A12831203195F286400831654
:100E70004908033C8A110A1283120319C62F640021
:100E800083164908043C8A110A1283120319682F39
:100E9000640083164908053C8A110A12831203195B
:100EA000532F8A01432E8A01EB218A017321831675
:100EB000AA011030AB004C30C50083128A015B23BD
:100EC00083164230C40083128A015C218A01432EBA
:100ED0008316F830C700C801B401B501B601B701E7
:100EE00083128A01EB218A0173218316AA01103033
:100EF000AB004C30C50083128A015B23831642305D
:100F0000C40083128A015C2183165108C20001309B
:100F1000B400B5018312831634088312A00083162F
:100F200035088312A100A30120308A01D1208A1143
:100F30000A12031DC42F83160130B600B7018312B5
:100F4000831636088312A000831637088312A10087
:100F5000A30180308A01D1208A110A12031DBB2F00
:100F60008A0153218316B60A0319B70A8A110A1295
:100F70008312031DA02F8316B40A0319B50A8A1120
:100F80000A128312031D8B2F8A01432E8A01EB2143
:100F90008A0173218316AA011030AB004C30C500C2
:100FA00083128A015B2383164230C40083128A01B4
:100FB0005C218316D90150088312A600A70183166D
:100FC0004F088312A200A3018A01E6208316BE0007
:100FD000831225088316BF000130BC00BD018312B7
:100FE00083163C088312A00083163D088312A100DB
:100FF00083163F088312A30083163E0883128A01DA
:10100000D1208A150A12031D5D280730BA0010305E
:10101000B8000730BB000830B900A0308A0150206A
:101020007F088A0150207E088A0150208A013520DD
:101030008316C0006400590850028A150A128312F0
:10104000031D412820308316AA070318AB0A463037
:10105000C40083128A015C2183162A08C20083120D
:101060008A01532183162B08C20083128A0153215F
:1010700083164C30C40083128A015C218316D90187
:10108000831283164230C40083128A015C218316C6
:101090004008831288000711000007158316D90A3B
:1010A0008312FE0A0319FF0A8316BC0A0319BD0A3C
:1010B0008A110A128312031DF02F8A01432E831610
:1010C000BE01BF01831211308A012F2011308A0125
:1010D0002F2011308A012F20E830AC000330AD0002
:1010E0008A0105208A110A12031C432E5D3C8A15D1
:1010F0000A12031D7028831641088312A9000530C7
:10110000B000B101A5013C308A0199208A110A1270
:10111000031C432E13308A012F2013308A012F2005
:1011200013308A012F208316C6018312FF308316E5
:1011300041078312B200FF300318013EB30083164B
:1011400046088312A000A1013308A30032088A01D7
:10115000D1208A150A12031DEC28831646083C3E4E
:10116000840000088312B200FF30A200A20A220805
:101170000F3C8A150A12031CE0288A150A12CC209B
:1011800032028A150A12031DB62822088316CE00E1
:1011900083128A150A12E02808308A002208820782
:1011A0003034313432343334343435343634373403
:1011B0003834393441344234433444344534463489
:1011C000831646083C3E84004E088000C60A8A15F5
:1011D0000A128312031D96288316C6018312FF305C
:1011E000831641078312B200FF300318013EB3009B
:1011F000831646088312A000A1013308A300320819
:101200008A01D1208A150A12031D61298316460816
:101210003C3E840000088312B2003208A000A10105
:1012200004308A01CC20B2002108B30001308316BB
:1012300046078312B400B501B50D34083C3E840066
:101240000008B400340832048316C2000730831249
:10125000BA001030B8000730BB000830B900A03029
:101260008A0150207F088A0150207E088A01502080
:101270008316420883128A014E2005308A01AC2071
:10128000FE0A0319FF0A8316BE0A0319BF0A3E08A5
:101290008312A00083163F088312A1007D08A300DB
:1012A0007C088A01D4208A150A12031D59298A0153
:1012B000432E02308316C6078A150A128312031CB6
:1012C000EF288A150A1263288A0173218316F830E1
:1012D000C700C801B401B501B601B701D901DA01EF
:1012E000003051078312B20010300318013EB300E2
:1012F000831652088312A600A7012030A200A30182
:101300008A01E620B4002508B500320834078316A8
:10131000AA00831233080318013E35078316AB0079
:101320004630C40083128A015C2183162A08C20059
:1013300083128A01532183162B08C20083128A016B
:10134000532183164C30C40083128A015C21113072
:101350008A012F2011308A012F2011308A012F207D
:10136000B830AC000B30AD008A0105208A110A129A
:10137000031C432E5D3C8A150A12031DB4298316F3
:1013800041088312A9000530B000B101A5013C302D
:101390008A0199208A110A12031C432E13308A01F4
:1013A0002F2013308A012F2013308A012F2083161B
:1013B000C6018312FF30831641078312B200FF304B
:1013C0000318013EB300831646088312A000A10152
:1013D0003308A30032088A01D1208A150A12031D9E
:1013E000302A831646083C3E840000088312B2006F
:1013F000FF30A200A20A22080F3C8A150A12031C21
:10140000242A8A150A12102232028A150A12031D92
:10141000FA2922088316CE0083128A150A12242A7A
:101420000A308A00220882073034313432343334AF
:101430003434353436343734383439344134423442
:101440004334443445344634831646083C3E8400D5
:101450004E088000C60A8A150A128312031DDA2973
:101460008316C6018312FF30831641078312B20030
:10147000FF300318013EB300831646088312A00014
:10148000A1013308A30032088A01D1208A150A126B
:10149000031DA72A831646083C3E840000088312D9
:1014A000B2003208A000A10104308A01CC20B200B1
:1014B0002108B3000130831646078312B400B5013A
:1014C000B50D34083C3E84000008B40034083204F2
:1014D0008316C0006400590850028A150A1283124C
:1014E000031D912A20308316AA070318AB0A463041
:1014F000C40083128A015C2183162A08C200831269
:101500008A01532183162B08C20083128A015321BA
:1015100083164C30C40083128A015C218316D901E2
:10152000831283164230C40083128A015C21831621
:101530004008831288000711000007158316D90A96
:101540000230C6078A150A128312031C332A8A1531
:101550000A12A7298A01432E63008A150A12AC2AAF
:02400E00753FFC
:00000001FF
